:100000002E288001840AFF3E031D01282928A30110
:10001000A200FF30A207031CA307031C29280330FA
:10002000A100DF3015200928A101E83EA000A109A8
:10003000FC30031C1E28A00703181B28A007000083
:10004000A10F1B2820182428A01C282800002828DD
:10005000080083138312031300000800FF23831694
:1000600090008312073099008501F93083168500CE
:10007000013096008B138B158113203084004030A3
:10008000831201200130A3002C30082085100508C0
:10009000A4000B10630085140A3007200518682897
:1000A00096300720051868280515A4013C30240265
:1000B000031864280330A300E8300820051C6128D9
:1000C0006428A40A031D5628051105186828652808
:0200D0004228C4
:02400E00843FED
:00000001FF
